:100000000C945D000C94CA010C947A000C947A0054
:100010000C947A000C947A000C947A000C947A0078
:100020000C947A000C947A000C947A000C947A0068
:100030000C947A000C947A000C947A000C947A0058
:100040000C947A000C947A000C947A000C947A0048
:100050000C947A000C947A000C947A000C947A0038
:100060000C947A000C947A000902120001010080BD
:100070001909040000000000000012011001FF0037
:100080000008C016DC050401010200010E03550042
:10009000530042006100730070001C03770077007A
:1000A00077002E00660069007300630068006C0032
:1000B0002E00640065000403090411241FBECFEF65
:1000C000D4E0DEBFCDBF11E0A0E0B1E0E0EFF2E1AF
:1000D00002C005900D92A230B107D9F711E0A2E05D
:1000E000B1E001C01D92AC34B107E1F70E94640990
:1000F0000C9476090C940000CF93DF936091280153
:10010000635067FD13C080912501CCE0D0E0C81B8F
:10011000D109C45DDE4F809124018D3209F458C0AD
:100120008091020187FD9DC01092280180910001FD
:1001300084FF41C0609101016F3F09F43CC0693008
:1001400008F470C06850609301018091180198E82C
:1001500089278093180168E08091020187FD1DC006
:10016000409126015091270186FF72C0FA01862F27
:10017000A9E1B1E094919D9331968150D9F7262F52
:10018000215030E02F5F3F4F240F351F3093270160
:1001900020932601C62FCC5F50C089E191E00E94D8
:1001A0002408682F893008F4A4C08FEF80930101E0
:1001B000CEE1C093000194E183B1837031F491509A
:1001C000D9F71092290110922301DF91CF91089560
:1001D000683009F0A9CF83EC809318018AE58093F9
:1001E0000001109202018881807609F045C09A8151
:1001F00010922101898181114AC01092220121E2CD
:1002000031E082E030932701209326018F3FC1F136
:100210009F81911104C09E81981708F4892F8093C3
:10022000010182CF109201018091180198E889277D
:1002300080931801611190CFC4E089E191E00E94A0
:10024000C601CC3009F4B5CF8FEF80930101B1CF57
:10025000DA01862FE9E1F1E09D9191938150E1F778
:100260008ECFCE010E9494088F3FF9F0882309F4C5
:100270005BCF1092010158CFCE010E947006C6CF0D
:10028000988197FD16C090E890930201C8CF853001
:1002900091F0863001F18830D1F0893091F021E27F
:1002A00031E08A3021F180E0ADCF8EE18093000112
:1002B0003BCF8E81E8CF9093290121E231E080E0AD
:1002C000A1CF90932B0121E231E080E09BCF2BE284
:1002D00031E081E097CF8B81813001F18230B1F044
:1002E000833051F080E090E4909302018FCF81E061
:1002F00089CFC82FCC5FA1CF911118C086EB90E0B9
:10030000909327018093260184E0EDCF88E690E06A
:10031000909327018093260182E1E5CF8AE790E060
:10032000909327018093260182E1DDCF913051F037
:100330009230C1F68CE890E09093270180932601DB
:100340008EE0D1CF8AE990E0909327018093260137
:100350008CE1C9CFE9E6F0E0808183608083E89A90
:100360000895A82FB92F80E090E041E050EA609511
:1003700030E009C02D9182279795879510F084274A
:100380009527305EC8F36F5FA8F30895EADF8D9379
:100390009D930895CF93CFB7CF93DF93C395189BC9
:1003A000E9F7189B11C0189B0FC0189B0DC0189B34
:1003B0000BC0189B09C0189B07C0189B05C0189B51
:1003C00003C0189B01C09CC05F93C0912501DD272D
:1003D000C45DDE4F2F9320E88894189B03C02F91B3
:1003E0005F91DFCF0F931F934F9312E06F933F9373
:1003F0003BE003B10370B1F1102710FD089427957D
:1004000000005FEF102FA8F7522703B14FEF10271E
:1004100010FB20F9122F197F39F1315020F1599337
:1004200013B10370F9F01370E9F0012700FB21F913
:10043000022F037F19F1000003B10370A1F0102710
:1004400010FB22F9122F177E11F100C0000013B12A
:10045000137049F0012700FB23F9022F0F7C01F1F3
:100460000000BEC02AC025C00370B9F2216013B1DC
:100470004E7F01270370B9F3012FCFCF03B1226064
:100480004D7F1027137079F3102F00C0D4CF246054
:100490004B7F13B10127037031F3012F00C0D5CF7B
:1004A0002860477F03B110271370E9F2102F00C0B6
:1004B000D7CF11E01CBB002717C03B503195C31BA1
:1004C000D04011E01CBB0881033CF9F00B34E9F08B
:1004D000209123011981110F1213EDCF093651F12B
:1004E0000D3211F0013E39F700932A013F916F91CF
:1004F0004F911F910F912F915F91CCB3C0FD4ECFC3
:10050000DF91CF91CFBFCF91189520912A0122235F
:1005100069F3109128011123D9F43430DAF03093C3
:10052000280120932401109125013BE0311B3093D9
:10053000250110C000912801013054F40AE53091E2
:10054000000134FD08C000930001C8E1D1E007C0FC
:100550004AE502C032ED432FC4E1D0E032E014B1ED
:100560001360289A05B114B910E053E020E860E464
:1005700020FF052705B927951795000000001C3FAF
:1005800020F56695A9F720FF0527279505B917954A
:100590001C3F00F529913A9551F70C7F10912901E4
:1005A000110F05B9C651D04011F01093230111E08D
:1005B0001CBB016014B11C7F402F4C7F54E05A9546
:1005C000F1F705B914B945B991CF052710E000C07E
:1005D00005B9D3CF052710E08894221FD6CF69CF65
:1005E00003B10370E1F3102710FB24F9122F1F79D8
:1005F00019F100C0000013B10000012700FB25F92C
:10060000022F0F7311F100C00000000003B110278A
:1006100010FB26F9122F1E7711F100C00000000018
:10062000000013B1012700FB27F9022F0C7F01F115
:100630004227542F0000E9CE20614F7E13B10127DD
:10064000037001F1012F00C0D4CF000020624F7D64
:1006500003B110271370B1F0102F0000D4CF00C0E9
:1006600020644F7B13B10127037061F0012FD5CFB8
:100670000000000020684F7703B11027137011F0BD
:10068000102FD6CFF0CE682F58E080E0709148014F
:100690002091470167FD1EC02B98660F880F1C999B
:1006A0008F5F2D9A36B5472F415030F096B5931B8A
:1006B0009217E0F34150D0F72D9836B5472F4150AF
:1006C00030F096B5931B9217E0F34150D0F751509C
:1006D00009F708952B9AE1CF8EBD0DB407FEFDCF2B
:1006E0008EB5089521E196958795779567952A951A
:1006F000D1F7209146012617D9F060934601E09189
:100700004301F09144018DE40995E0914301F0919A
:10071000440180E00995E0914301F091440180910A
:1007200046010995E0914301F091440180E009946C
:100730000895809145018CBD809142018DBD089541
:100740008823B1F0893008F04AC023E433E03093C5
:1007500044012093430191E090934801853001F1D9
:10076000C0F08730A1F168F589E0809347010895D2
:100770008CE693E0909344018093430110924201F0
:1007800081E0809347018093480182E58093450191
:100790000895833001F140F084E280934701089589
:1007A00082E1809347010895823039F080E9809397
:1007B000470182E080934801089580E980934701D2
:1007C0000895883099F782E080934701089585E085
:1007D00080934701089588E48093470108952CE6AB
:1007E00033E030934401209343011092420191E0A1
:1007F0009093470190934801893049F030F28B3053
:1008000051F08C3011F681E580934501089583E520
:1008100080934501089582E58093450190934201BC
:10082000089526B53091480190914701315030F03C
:1008300086B5821B8917E0F33150D0F7089584B153
:100840008C6284B92A982D9826B530914801432F9F
:1008500090914701415030F086B5821B8917E0F333
:100860004150D0F72A9A26B5315030F086B5821B18
:100870008917E0F33150D0F72A9880914301909185
:1008800044018C56934019F01092460108958091CE
:1008900045018CBD809142018DBD109246010895A5
:1008A00084B1837D84B985B1837D85B91CBC0895ED
:1008B000CF93DF93C0E2E0914301F09144018CEAD1
:1008C0000995E0914301F091440183E50995E09198
:1008D0004301F091440180E00995D82FE091430154
:1008E000F091440180E00995D33509F43AC01CBC6D
:1008F00026B530914801432F90914701415030F087
:1009000086B5821B8917E0F34150D0F72A9A26B5A5
:10091000432F415030F086B5821B8917E0F34150D8
:10092000D0F72A9826B5315030F086B5821B89174A
:10093000E0F33150D0F7E0914301F091440183E0BE
:10094000EC36F80739F0C15009F0B9CF81E0DF91FA
:10095000CF910895809145018CBD809142018DBD5C
:10096000F2CF80E0DF91CF910895CF92DF92EF92A6
:10097000FF926B017C010E947203D701C601817056
:100980009927AA27BB27880F880F880FE09143017A
:10099000F091440180620995D701C60139E0B6950E
:1009A000A795979587953A95D1F7E0914301F091F6
:1009B00044010995D701C601B695A79597958795E6
:1009C000E0914301F09144010995E0914301F091D8
:1009D000440180E0FF90EF90DF90CF900994CF9298
:1009E000DF92EF92FF920F931F93CF93DF936B01F0
:1009F0007C01C42FD22F0E947203970186010170DF
:100A0000112722273327802F880F880F880FE09126
:100A10004301F091440180640995D701C60159E072
:100A2000B695A795979587955A95D1F7E09143018B
:100A3000F09144010995D701C601B695A795979500
:100A40008795E0914301F09144010995E0914301BC
:100A5000F09144018C2F0995DD23B9F0CF3791F047
:100A6000D6B5CEE1C701B6010E94B5048F3769F44F
:100A700086B58D1B8B3510F0D6B5C150C111F2CFA4
:100A800081E004C08FE00E94FB0580E0DF91CF9100
:100A90001F910F91FF90EF90DF90CF900895CF922C
:100AA000DF92EF92FF920F931F93CF93DF931F92EA
:100AB000CDB7DEB76B017C0149830E947203E091E0
:100AC0004301F09144018CE40995D701C60179E016
:100AD000B695A795979587957A95D1F7E0914301BB
:100AE000F09144010995D701C601B695A795979550
:100AF0008795E0914301F09144010995E09143010C
:100B0000F091440180E0099549814F3FE9F006B535
:100B10001EE1C701B6010E94B5048F3F99F486B566
:100B2000801B8B3510F006B511501111F2CF81E00A
:100B30000F90DF91CF911F910F91FF90EF90DF9079
:100B4000CF90089580E0F4CF8FE00E94FB0580E015
:100B5000EFCF1F93CF93DF931F92CDB7DEB7182F40
:100B6000E0914301F091440180EA99830995E09175
:100B70004301F09144019981892F0995E091430146
:100B8000F0914401812F0995E0914301F0914401D6
:100B900080E00F90DF91CF911F9109941F93CF9325
:100BA000DF9300D0CDB7DEB7182FE0914301F0916D
:100BB000440180EC6A8399830995E0914301F091A7
:100BC00044019981892F0995E0914301F0914401F5
:100BD000812F0995E0914301F09144016A81862FAC
:100BE00009958EE10E94FB0580E00F900F90DF9148
:100BF000CF911F910895882349F030E026B596B52E
:100C0000921B9A35E0F33F5F3813F8CF0895259A89
:100C100023982B9A50E217D05A95E9F70895AC0122
:100C200088E605D0842F03D089E601D0852F0FD028
:100C300028E030E0382780FB869506D02A95D1F74A
:100C400030FB02D000D0689423982B9A16F02B9892
:100C5000239AE0914A01F0914B013197F0F72D9AD8
:100C6000E3B1E3FBE0914A01F0914B013197F0F7DA
:100C70002D98089520ECE7DF46F42A95E1F780E00F
:100C80002AE1E5DF2A95E9F7DECF28E030E0DBDF77
:100C9000869587F938272A95D1F7D5DF27F93227A6
:100CA00072F3D1DFD0CFDB01742FB9DF84E2BFDF75
:100CB000E1DF8D937A95D1F70895DB01742FAFDFD3
:100CC00083EFB5DF8DE1B3DF84E6B1DF8D91AFDF78
:100CD00082E7ADDFCFDF8078D9F77A9589F708957D
:100CE000CF93DF93EC018981813089F1823009F45F
:100CF000ABC0833009F461C08430B1F1873009F4AE
:100D000082C0853009F402C1863009F4A2C088305F
:100D100009F4D5C0893009F4FFC08A3009F42AC12A
:100D20008B3009F456C18C3009F469C18D3009F457
:100D300080C18E3009F483C18F3009F4FEC0803148
:100D400009F41FC18F3709F439C180E02DC0329BEF
:100D500056C0809103010E94A003109204014198A3
:100D60000E941F0480E020C080910401811110C006
:100D70005B8140E08A81482B662757FD6095762F7E
:100D800040930D0150930E0160930F017093100179
:100D90009F8180E02E81822B90931201809311011C
:100DA00082E0809313018FEF25E031E0309327013B
:100DB00020932601DF91CF910895E0914301F091B6
:100DC00044018A81099580930501E0914301F091E6
:100DD00044018B81099580930601E0914301F091D4
:100DE00044018C81099580930701E0914301F091C2
:100DF00044018D8109958093080184E0D5CF85E079
:100E00000E94A003AACF80910401811110C05B81D0
:100E100040E08A81482B662757FD6095762F4093E6
:100E20000D0150930E0160930F01709310019F818B
:100E300080E02E81822B909312018093110183E038
:100E4000809313018FEFB0CF0E945004419A80E04D
:100E5000ABCF80910401811110C09B8180E02A8179
:100E6000822BAA2797FDA095BA2F80930D0190930E
:100E70000E01A0930F01B09310013C812D81822FB0
:100E80008F7080931601822F807F40E1849FC00184
:100E90001124830F911D909315018093140120FD5F
:100EA000809317019F8180E02E81822B9093120105
:100EB0008093110181E0809313018FEF75CF8091B2
:100EC0000401811110C09B8180E02A81822BAA2716
:100ED00097FDA095BA2F80930D0190930E01A093DA
:100EE0000F01B0931001109215011092140110928D
:100EF00016019F8180E02E81822B909312018093B6
:100F0000110184E0809313018FEF4ECF0E945804AB
:100F10008093050181E048CF81E0809304018A81BC
:100F20009B81AC81BD8180930D0190930E01A093B4
:100F30000F01B093100180E037CF9B8180E02A81C0
:100F4000822BAA2797FDA095BA2F80930D0190932D
:100F50000E01A0930F01B09310019F8180E02E81BC
:100F6000822B909312018093110185E080931301ED
:100F70008FEF1ACF8A81809303011092050181E0DF
:100F800013CF9B8180E02A81822BAA2797FDA09511
:100F9000BA2F80930D0190930E01A0930F01B0938F
:100FA00010019F8180E02E81822B9093120180930B
:100FB000110186E0809313018FEFF6CE81E08093DC
:100FC000050110920601109207011092080184E0B9
:100FD000EBCE9B8180E02A81822B90934B01809302
:100FE0004A012A9A229A83E00E94FB052A98419896
:100FF00080E10E94FB050E94070680E0D5CE80ECD0
:101000000E94170680E00E9417068AE00E94FB05F6
:101010002A9A85E00E94FB052A9885E00E94FB053C
:1010200084B1837D84B985B1837D85B9419A80E09F
:10103000BBCE0E943A068093050181E0B5CE8A813D
:101040000E94170680E0B0CE0F931F93CF93DF93DB
:10105000582F792F062F20911301322F3250323022
:1010600050F0253009F443C00FEF802FDF91CF916E
:101070001F910F910895662391F180910D01909138
:101080000E01A0910F01B0911001C52FD72F10E0D4
:101090001CC00E94A905888380910D0190910E01CA
:1010A000A0910F01B09110010196A11DB11D809377
:1010B0000D0190930E01A0930F01B09310011F5FDB
:1010C0002196101751F020911301223011F7BC0125
:1010D000CD010E94B5048883DFCF083030F610922E
:1010E0001301802FDF91CF911F910F910895462F0B
:1010F000682F80910D0190910E010E9453068091FE
:101100000D0190910E01A0910F01B0911001800F7F
:10111000911DA11DB11D80930D0190930E01A0930F
:101120000F01B0931001A1CFFF920F931F93CF93A4
:10113000DF93382F792F162F20911301213071F072
:10114000243061F0263009F490C0FF24FA948F2DEA
:10115000DF91CF911F910F91FF900895112309F412
:10116000B1C080910D0190910E01A0910F01B0913D
:101170001001C32FD72F00E0F12C50C02091140193
:1011800030911501232B09F053C021E04881BC01A7
:10119000CD010E94EF0420911101309112012150E4
:1011A00031093093120120931101232BE9F410929D
:1011B00013018091160181FF38C02091170130E0A2
:1011C00080911401909115012817390771F16091F0
:1011D0000D0170910E0180910F01909110014881D5
:1011E0000E944F05FF24F39480910D0190910E0110
:1011F000A0910F01B09110010196A11DB11D809326
:101200000D0190930E01A0930F01B09310010F5F99
:101210002196011709F49BCF20911301213009F485
:10122000ADCF68810E94CE05B6CFFF24F394DCCF0A
:1012300020E04881BC01CD010E94EF04809117019C
:101240008150809317018111A6CF60910D0170919B
:101250000E0180910F019091100148810E944F056D
:10126000809114018093170196CF462F682F8091AB
:101270000D0190910E010E945D0680910D019091EB
:101280000E01A0910F01B0911001810F911DA11DC0
:10129000B11D80930D0190930E01A0930F01B093A7
:1012A00010018091110190911201811B910990937D
:1012B000120180931101892B29F410921301FF244C
:1012C000F39445CFF12C43CF1BB815B88BEF8AB9F7
:1012D0008FEF84B914B883E087B99EEF98B985BDC4
:1012E0000E94AA0178940E947C00FDCFF894FFCF61
:0212F0005AFFA3
:00000001FF
